:020000040000FA
:10000000F00200106901000071010000730100009E
:100010007501000077010000790100000000000078
:100020000000000000000000000000007B01000054
:100030007D010000000000007F0100008101000040
:1000400083010000830100008301000083010000A0
:100050008301000083010000830100008301000090
:100060008301000083010000830100008301000080
:100070008301000083010000830100008301000070
:100080008301000083010000830100008301000060
:100090008301000083010000830100008301000050
:1000A0008301000083010000830100008301000040
:1000B0008301000083010000830100008301000030
:1000C00083010000830100008301000000F002F8BA
:1000D00000F03AF80AA090E8000C82448344AAF1A8
:1000E0000107DA4501D100F02FF8AFF2090EBAE8A6
:1000F0000F0013F0010F18BFFB1A43F0010318475C
:100100004408000064080000103A24BF78C878C191
:10011000FAD8520724BF30C830C144BF04680C600D
:10012000704700000023002400250026103A28BF55
:1001300078C1FBD8520728BF30C148BF0B60704759
:100140001FB51FBD10B510BD00F0A6F81146FFF792
:10015000F7FF00F0C6FA00F0C4F803B4FFF7F2FFAF
:1001600003BC00F0E9FB000009488047094800474C
:10017000FEE7FEE7FEE7FEE7FEE7FEE7FEE7FEE757
:10018000FEE7FEE704480549034A054B70470000B7
:10019000A9040000CD000000F0000010F0020010E3
:1001A000F000001053EA020C00F069802DE9F04BDA
:1001B0004FF00006002B1FBFB3FA83F503FA05F4D6
:1001C00024FA05F65E4012BF1643B2FA82F502FA2F
:1001D00005F4C5F120051EBF22FA05FC44EA0C0413
:1001E000203556EA044C4FEA144418BF641C4FF003
:1001F00000084FF00009904271EB030C39D300293D
:1002000019BFB1FA81F701FA07F6B0FA80F700FAE0
:1002100007F6C7F120071EBF20FA07FC46EA0C06C6
:100220002037B6FBF4FCA7EB0507103F07F01F0BC8
:10023000CBF120060CFA0BFB2CFA06F644BFB346B2
:100240000026202FA4BF5E464FF0000B5BEA060C91
:1002500008BF4FF0010B19EB0B09ABFB027C48EB1D
:100260000608C01B06FB02CC0BFB03CC71EB0C0198
:10027000C1E70B46024641464846BDE8F08B13B540
:100280004FF000004FF00001AFF30080BDE81C40CC
:100290007047704770477047754600F029F8AE46C2
:1002A00005006946534620F00700854618B020B582
:1002B000FFF768FFBDE820404FF000064FF0000751
:1002C0004FF000084FF0000B21F00701AC46ACE8FE
:1002D000C009ACE8C009ACE8C009ACE8C0098D466B
:1002E00070470446AFF300802046FFF736FF00005A
:1002F000004870479000001070470000FFFFFFFFAC
:100300002DE9F04781480068C0F3016003287CD1E3
:100310007F48006810F0030006D0012833D002287F
:100320005FD003282ED100E000BF78480068C0F3FA
:10033000074000F101044FF002017648D0F8880030
:10034000C0F30E0000F10100A1FB0001724B4FF061
:10035000000CA0FB037901FB039100FB0C1122466A
:1003600063463846FFF71EFF05466C480068C0B27A
:1003700000F1010422464FF000032846FFF712FF68
:10038000674908605DE061480068C0F3074000F11C
:1003900001044FF002015F48D0F88800C0F30E005E
:1003A00000F10100A1FB00105E4A4FF0000CA1FB20
:1003B000027900FB029001FB0C012246634638469D
:1003C000FFF7F0FE054655480068C0B200F1010491
:1003D00022464FF000032846FFF7E4FE504908602C
:1003E0002FE04A480068C0F3074000F101044FF0D5
:1003F00002014848D0F88800C0F30E0000F1010067
:10040000A1FB00124FF4004000E01BE04FF000039E
:10041000A1FB007902FB009001FB03012246384654
:10042000FFF7C0FE05463D480068C0B200F1010478
:1004300022464FF000032846FFF7B4FE3849086013
:1004400000BF2FE03248006810F0030006D00128FA
:1004500010D0022819D0032823D100E000BF2F4874
:100460000068C0B200F101002B49B1FBF0F02C494B
:10047000086016E029480068C0B200F1010029496F
:10048000B1FBF0F0264908600BE024480068C0B2D8
:1004900000F101004FF40041B1FBF0F02049086089
:1004A00000BF00BFBDE8F08720201F490860194841
:1004B000D0F8A00110F0200F05D000BF1A48006846
:1004C00010F0400FFAD00320144908601748114972
:1004D000C1F8A8011648174908604FF001000C49FF
:1004E00008604FF00400A1F10401086012481349AC
:1004F00008604FF480700749C1F8C80108460068D9
:1005000020F4704040F480400860704788C00F407D
:100510000CC10F4000C00F4000093D0004C10F4056
:1005200000000010001BB700A0C10F4055515155ED
:1005300055545554ACC10F40DEF7EFEFC4C00F4027
:10054000002100E0491C8142FCD3704700B5002027
:10055000E5494861E54800684861E548007818B910
:100560004FF00060C86103E04FF00060DE49886131
:100570004FF08050DC4988611920FFF7E1FF4FF010
:100580008050D949C86141F28830FFF7D9FF00BDDA
:1005900000B5D7480078012801D100200AE0D548ED
:1005A0000068302803D0D3480068202801D10120FA
:1005B00000E00020D0490870CE48007800F0F0003C
:1005C000CA49086008460088C0040860FFF7BEFFFB
:1005D000C948007858B9C748007800F00F00C349EF
:1005E000086008460088C0050860FFF7AFFF00BD3F
:1005F000BD48406BC14908600846006800F0F060E3
:1006000008600846006828B30120BD490870BB484F
:100610000068B0F5000F03D10020BA49087019E056
:10062000B6480068B0F1807F03D10120B549087059
:1006300010E0B2480068B0F1007F03D10220B14958
:10064000087007E0AD480068B0F1806F02D1032068
:10065000AC490870704700B542E00020AA49087014
:100660003AE0A948007820B94FF48060A7490860B3
:1006700017E0A5480078012803D1C002A34908600B
:100680000FE0A1480078022803D1C0029F4908600A
:1006900007E09D480078032803D14FF400509B49A0
:1006A00008609A480068904948650020944908709D
:1006B000FFF79EFF92480078012808D1944892499C
:1006C000097800EB81008F490978405C00BD8E48B5
:1006D0000078401C8C4908708B4800780428C0DBE7
:1006E000BBE710B5FFF7E0FEFFF70AFE4FF0FC5046
:1006F0007D490860002008624FF4705008640020B3
:100700007B490870834908600DE083488149096886
:1007100050F8210077490860FFF73AFF7D480068EC
:10072000401C7C4908607B4800680928EDD3012003
:100730006F490870FFF78FFF784908700846007806
:100740006C490860FFF724FF7548FFF7F9FE0020A9
:10075000674908707048C06966490860FFF718FF6C
:10076000012063490870FFF776FF6E4908706B48F7
:1007700000786D4908706B480078487000208870D8
:10078000644908600CE0684862490968405C59495E
:100790000860FFF7FDFE5F480068401C5D49086087
:1007A00061485C490968405C0028ECD15C48FFF76F
:1007B000C7FE00204E4908705748C0694D4908607F
:1007C000FFF7E6FE01204A490870FFF744FF57494A
:1007D00008705248007854490870524800784870B0
:1007E0005248007888700020C8704A4908600CE0C0
:1007F0004D4848490968405C3E490860FFF7C8FE1B
:1008000044480068401C434908604748414909681A
:10081000405C0028ECD14248FFF792FE00203449AA
:1008200008703D48C06933490860FFF7B1FE0120F8
:100830002F490870FFF70FFF3D49087037480078CF
:10084000394908703748007848703848007888700F
:1008500037480078C870364800783D281AD13148AA
:1008600000782B2802D02D2812D108E02B480078E0
:100870002E490978084430382E49087009E0274885
:1008800000782A490978401A30302A49087000E077
:1008900000BF00BF27480078234908710020487135
:1008A0001C4908600CE020481A490968405C11495D
:1008B0000860FFF76DFE17480068401C1549086086
:1008C000194814490968405C0028ECD11448FFF726
:1008D00037FE0020064908700F48C06905490860C6
:1008E000FFF756FE002010BD00C0092008000010D0
:1008F0000C000010040000100D0000106400001037
:100900005B000010590000105A0000106000001039
:1009100038000010480000101000001054000010B3
:1009200020A10700560000108000001055000010A4
:10093000570000105800001001491820ABBEFEE718
:100940002600020064090000000000108000000082
:1009500008010000E409000080000010700200009F
:1009600024010000C0C62D000000000000000000AF
:1009700000000000300000003000000030000000E7
:1009800020000000280000000C000000060000000D
:100990000100000080000000000000003031323310
:1009A0003435363738392B2D2A2F3D3D00000000D5
:1009B0000000000000000000000000000000000037
:1009C0000000000000000000000000000000000027
:1009D0000000000000000000000000000000000017
:0409E0000000000013
:04000005000001698D
:00000001FF
